:100000000C94AA020C94E2020C94E2020C94E20218
:100010000C94E2020C94E2020C94E2020C94E202D0
:100020000C94E2020C94E2020C940E250C94E02550
:100030000C940B200C94E2020C94E2020C94E20269
:100040000C94E2020C94E2020C94E2020C94E202A0
:100050000C94E2020C9493200C94E2020C94E202C1
:100060000C94E2020C94E2020C94E2020C94E20280
:100070000C94E2020C94E2020C94E2020C94E20270
:100080000C94E2020C94E2020C94E2020C94E20260
:100090000C94E2020C94E2020C94E2020C94E20250
:1000A0000C94E2020C94E2020C94E202A105A10578
:1000B000CD05CD0535066007600760075306EC06E1
:1000C000FD06FD064D2674266C2774266C27C02677
:1000D000E3266C273A27492729001E001F0020002D
:1000E00021002200230024002500260027002D00E7
:1000F0002E0000002A0035002B0014001A00080012
:10010000150017001C0018000C00120013002F002F
:100110003000000031004C003900040016000700D8
:1001200009000A000B000D000E000F003300340020
:100130000000000028004B00E10000001D001B0033
:1001400006001900050011001000360037003800C5
:10015000E500000052004E00E000E300E200000075
:100160000000000000002C0000000000E60001512B
:100170005000000051004F0035003A003B003C00A9
:100180003D003E003F00400041004200430044006B
:100190004500000046000100C35CCA5CC85CC65C48
:1001A000005C0100010001000100010001000100EC
:1001B00001000000010049000100CB5CC95CC75C84
:1001C0000100010001000100010001000100010027
:1001D0000000000001004A000100000001000100D1
:1001E000010001000100010001000100BE5CBF5CD4
:1001F000A8000000A9004D0001000100010000005E
:10020000000000000000C05C0000000001000100D0
:1002100001000000AA00010000047F3F1F643214A7
:10022000643214783C1E1E140A0522232526282930
:100230002A2C2D2F3032333536383A3B3D3E404262
:10024000434547494A4C4E5051535557595A5C5EA5
:100250006062646668696B6D6F71737577797B7DB9
:100260007F81838587898A8C8E90929496989A9CB8
:100270009E9FA1A3A5A7A8AAACAEAFB1B3B4B6B8D0
:10028000B9BBBCBEBFC1C2C3C5C6C7C9CACBCCCD32
:10029000CED0D1D2D2D3D4D5D6D7D7D8D9D9DADA0D
:1002A000DBDBDBDCDCDCDCDCDDDDDDDDDCDCDCDC8D
:1002B000DCDBDBDBDADAD9D9D8D7D7D6D5D4D3D2C1
:1002C000D2D1D0CECDCCCBCAC9C7C6C5C3C2C1BF9F
:1002D000BEBCBBB9B8B6B4B3B1AFAEACAAA8A7A503
:1002E000A3A19F9E9C9A98969492908E8C8A8987BF
:1002F0008583817F7D7B79777573716F6D6B69689D
:10030000666462605E5C5A5957555351504E4C4A70
:100310004947454342403E3D3B3A3836353332301B
:100320002F2D2C2A292826252322FFAA7F5540007D
:1003300001010101010101010102020202020202A6
:100340000202030303030303030304040404040479
:10035000040505050505060606060607070707073F
:1003600008080808090909090A0A0A0B0B0B0C0CF2
:100370000C0D0D0D0E0E0E0F0F0F1010111111128E
:100380001213131414151516161717181819191A0D
:100390001A1B1B1C1D1D1E1E1F2020212222232470
:1003A00024252626272829292A2B2C2D2D2E2F30AF
:1003B000313232333435363738393A3B3C3D3E3FC3
:1003C000404142434445464748494A4C4D4E4F50B0
:1003D000515354555658595A5B5D5E5F616264656E
:1003E0006668696B6C6D6F7072737577787A7B7DF8
:1003F0007E8082838587888A8C8E8F91939596984C
:100400009A9C9EA0A2A3A5A7A9ABADAFB1B3B5B767
:10041000BABCBEC0C2C4C6C9CBCDCFD1D4D6D8DB3E
:10042000DDDFE2E4E7E9EBEEF0F3F5F8FAFDFF14C7
:10043000033200360038002E0032005F00520047C1
:1004400000420000000E034E006F00780061007251
:1004500000790000000403090409023B00020100C6
:10046000A0FA0904000001030101000921110100A3
:100470000122400007058103080001090401000171
:1004800003000000092111010001226D000705820F
:10049000032000011201000200000008584E7C0AEF
:1004A00001000102000105010980A1018503190174
:1004B0002AB700150126B700950175108100C00507
:1004C0000C0901A101850419012AA002150126A029
:1004D00002950175108100C005010906A10185067C
:1004E000050719E029E71500250195087501810226
:1004F0000507190029EF1500250195F07501810206
:1005000005081901290595057501910295017503E5
:100510009101C005010906A101050719E029E715A8
:100520000025019508750181029501750881010575
:1005300007190029FF150026FF00950675088100A0
:1005400005081901290595057501910295017503A5
:100550009101C00011241FBECFEFDAE0DEBFCDBF96
:1005600004B603FE18C080912A0390912B03A0913A
:100570002C03B0912D038730904BA740B04B59F41A
:1005800010922A0310922B0310922C0310922D0329
:10059000E0E0F8E3099511E0A0E0B1E0EAE2F1E57E
:1005A00002C005900D92A03CB107D9F723E0A0EC62
:1005B000B1E001C01D92AA32B207E1F70E945E13BA
:1005C0000C9493280C94000081E0089581E0089534
:1005D0000C94E60208950C94EA021F93CF93DF93E4
:1005E00000D000D01F92CDB7DEB749835A836B830A
:1005F0003091C30189819A81311114C0662359F069
:10060000222349F00E949909182F682F89819A8125
:100610000E94420903C00E946D09182F69817A81E6
:10062000812F04C00E94990969817A810F900F90EF
:100630000F900F900F90DF91CF911F910C94C710E6
:10064000FC01262F408151816281738184810C9449
:10065000ED0281E00895CF93DF93EC0160E00E940A
:100660002003BE01DF91CF910C94EB020C940F128A
:100670000C940B1208950E94EC070E943A032FEF8E
:1006800084E39CE0215080409040E1F700C00000EE
:100690000C94B9200F931F93CF93DF938C0161E0EB
:1006A0000E942003EC01B8010E94E802882309F4AB
:1006B0004BC0B801CE010E94521B882309F444C0EC
:1006C000B801CE010E94641E8823F1F1B801CE0169
:1006D0000E94781C8823C1F1B801CE010E94C01D80
:1006E000882391F1B801CE010E949619882361F107
:1006F000F8018281882309F1CB358DE5D807C1F057
:1007000050F4C115FCE5DF0781F0CF3DDC45A9F4CD
:100710000E94D00E19C0CC35EDE5DE0761F0CD3575
:10072000DD4559F40E94130E08C00E943B030CC023
:100730000E941C0E02C00E941F0EC801DF91CF91C3
:100740001F910F910C94E40280E0DF91CF911F91F3
:100750000F9108950E94ED1F80E00E94871B0C946A
:10076000D5030E94761A0E94D8030C94F31F0895B3
:100770000C94B70381E00895CF93C82F0E94BA0369
:10078000882329F0C1FF02C0289A01C02898CF9180
:100790000895209A28980895CF93C82F0E94B803EF
:1007A0008C2F0E94BC03CF91089580E00C94CC0361
:1007B0000E94C01E0C94CC030E94C01E9091C201E6
:1007C000891721F08093C2010C94CC030895CF9334
:1007D000DF93CDB7DEB72B970FB6F894DEBF0FBE11
:1007E000CDBF4F83588769877A878B8761110E94B5
:1007F0005F0D9E012F5F3F4F86E0F90111928A95B0
:10080000E9F785E0FE013796D90101900D928A95AE
:10081000E1F789819A814C815D81452B31F09F3FC1
:1008200031F491E08F3F19F403C091E001C090E0F2
:1008300090FF09C049815A816B817C818D819E81A5
:100840000E94800C05C0C9010E9429038111F2CFCA
:100850002B960FB6F894DEBF0FBECDBFDF91CF91C0
:100860000895FC01808191810E94DB090895CF9356
:10087000882309F49CC0C82F8238C1F40E94C01E8E
:1008800081FD95C069E380910201909103010E946E
:10089000A81F0E94810D2FEF81EE94E0215080402F
:1008A0009040E1F700C0000069E319C0833801F50A
:1008B0000E94C01E80FD7BC063E580910201909183
:1008C00003010E94A81F0E94810D2FEF81EE94E08A
:1008D000215080409040E1F700C0000063E5809126
:1008E0000201909103010E94B31FCF910C94810DDE
:1008F0008438C1F40E94C01E82FD59C067E4809113
:100900000201909103010E94A81F0E94810D2FEF08
:1009100081EE94E0215080409040E1F700C000005B
:1009200067E4DDCF8CEF8C0F813AD0F46C2F80918F
:100930000201909103010E94281F882349F06C2F27
:1009400080910201909103010E94B31F0E94810DCA
:100950006C2F80910201909103010E94A81FC5CFC6
:1009600080E28C0F883048F4C77081E001C0880FA6
:10097000CA95EAF70E94420DB8CFEBE5EC0FE330E1
:1009800040F4F0E0EE5AFE4F808190E0CF910C945D
:10099000E61EC85AC73158F4EC2FF0E0EE0FFF1FE7
:1009A000EC5DFE4F80819181CF910C94FC1ECF9124
:1009B0000895882309F45BC0682F823879F40E9477
:1009C000C01E81FF54C069E3809102019091030130
:1009D0000E94A81F0E94810D69E310C08338B1F402
:1009E0000E94C01E80FF43C063E580910201909188
:1009F00003010E94A81F0E94810D63E580910201FE
:100A0000909103010E94B31F0C94810D843879F4F6
:100A10000E94C01E82FF2BC067E48091020190916A
:100A200003010E94A81F0E94810D67E4E7CF8CEFAD
:100A3000860F813A18F380E2860F883048F4677099
:100A400081E001C0880F6A95EAF70E94480DDCCF6B
:100A50008BE5860F833020F480E090E00C94E61E56
:100A6000685A673120F480E090E00C94FC1E0895F1
:100A70001F93CF93DF93182FEB010E943704209729
:100A800041F08FE99FE00197F1F700C00000219746
:100A9000F6CF812FDF91CF911F910C94D904893328
:100AA00019F060E070E002C060E570E00C94380579
:100AB000882321F00E94420D0C94810D0895882313
:100AC00021F00E94480D0C94810D0895CF92DF9281
:100AD000EF92FF920F931F93CF93DF937C01D62F5A
:100AE000C72FFC011281058102950F700E94380DFD
:100AF0008823B9F01123A9F08C2F807F803421F056
:100B000080E28D0F883068F08091CE0282FD09C0AE
:100B100082E00E94E10D0E94380D91E0D82ED92686
:100B200001C0D12CCC2EC2948FE0C8228C2D90E035
:100B30008C30910508F0C4C1FC01EA5AFF4F0C94B7
:100B4000FA278C2F807FCF70882311F0C295C07F49
:100B5000112399F0CC2309F49FC180E28D0F8830D6
:100B600010F0D11104C08C2F0E94420D03C08C2FB5
:100B70000E94520D0E94810D8FC18D2F0E94D904B9
:100B8000CC2309F49DC180E28D0F883038F1DD233C
:100B900029F18C2F0E94580D24C08C2F807FCF709C
:100BA000803211F0C295C07FDD2319F0D130A1F160
:100BB0003DC08091CE0282FF17C0112349F0CC23A3
:100BC00029F08C2F0E94420D0E94810D80E065C1AA
:100BD00080E00E94D904CC2309F472C18C2F0E94BA
:100BE000480D0E94810D6CC1112371F0002341F06A
:100BF000013031F40E94620D8C2B0E946A0D60C19D
:100C00000E94620D8C2B1DC0002319F0013009F4E5
:100C100057C10E94770D25C0112321F0063008F03E
:100C20004FC10EC0053008F04BC11BC0112361F04D
:100C3000002331F0F701858180FF2EC18F708583FD
:100C40008C2F0E9458053CC1002359F0D93309F07C
:100C500034C1FFEF07EE13E0F15000401040E1F720
:100C60002AC18C2F0E945F052BC18C2F86958695FB
:100C7000837019F0813061F023C1112321F08D2F91
:100C80009C2F937002C080E090E00E94E61E20C17D
:100C9000112321F08D2F9C2F937002C080E090E0F3
:100CA0000E94FC1E15C18C2F837009F047C01111E2
:100CB0000BC12D2F229526952770220F220F6D2F05
:100CC0006F70862F90E0A0E0B0E0022E04C0880F85
:100CD000991FAA1FBB1F0A94D2F7D4FF10C04FE080
:100CE00050E060E070E004C0440F551F661F771F9E
:100CF0002A95D2F7409550956095709503C040E0D5
:100D000050E0BA01C695C695C3708A019B01082BB5
:100D1000192B2A2B3B2BC901B801C23049F058F4DA
:100D2000C13019F00E945808CFC00E944608CCC0BC
:100D30000E946A08C9C00E944408C6C0112319F065
:100D40008C2F817001C08695882309F4BDC02D2F9A
:100D5000229526952770220F220F6D2F6F70862FF8
:100D600090E0A0E0B0E0022E04C0880F991FAA1FF7
:100D7000BB1F0A94D2F7D4FF10C04FE050E060E0F0
:100D800070E004C0440F551F661F771F2A95D2F7E5
:100D9000409550956095709503C040E050E0BA01D1
:100DA000C695C695C3708A019B01082B192B2A2B67
:100DB0003B2BC901B801C23049F058F4C13019F0D9
:100DC0000E941D0981C00E940B097EC00E942F094C
:100DD0007BC00E947E0878C0CF70112339F08C2F21
:100DE0000E94A4088D2F0E9458056EC08D2F0E946E
:100DF0005F058C2F0E94C50867C0D23F21F128F4FF
:100E0000D03F41F0D13FC1F043C0D33F19F1D43FAF
:100E100079F03EC0112341F0053008F051C08C2F0D
:100E20008F710E94EA084CC0063008F049C0F7CF25
:100E30008091CE0282FF18C0112339F08C2F8F7160
:100E40000E94A4083DC01123C9F38C2F8F710E940A
:100E5000C50836C0112329F08C2F8F710E948F088E
:100E60002FC00E948A082CC0112349F0CF718C2F0B
:100E70000E94A40863E08C2F0E94C60D21C081E06F
:100E80000E94E10D0230E0F082E00E94E10D18C006
:100E9000112331F0002391F28D2F0E94370410C0EE
:100EA000002399F2D93349F41FEF27EE33E01150B4
:100EB00020403040E1F700C000008D2F0E94D9048F
:100EC00088EF8C0D843020F40E94C01E0E94CC0359
:100ED000DD20C9F00E94340D80FD15C0F70112829B
:100EE0000E942E0D0E94A408C7010E94A4070E9420
:100EF0002E0DDF91CF911F910F91FF90EF90DF901A
:100F0000CF900C94C508DF91CF911F910F91FF9066
:100F1000EF90DF90CF9008950F931F93CF93DF93BF
:100F2000EC01688179818A810E94E6098C010E9426
:100F300041090E943208B801CE010E946605DF9186
:100F4000CF911F910F910895CF93DF93EC0198817A
:100F500089812B813C81232B31F08F3F31F481E05B
:100F60009F3F19F403C081E001C080E080FD1DC0F7
:100F7000CE010E944A03811110C00E94380D8823BF
:100F8000A1F08A81882389F08091CE0282FD0DC074
:100F900082E0DF91CF910C94E10DCE010E948C078D
:100FA000CE01DF91CF910C942B03DF91CF91089567
:100FB00080E090E00E94E61E80E090E00E94FC1E2F
:100FC0000E945F0D0C94810D8091020190910301AC
:100FD0000E94BE1F0C94D8070E944F0D0C94E4078A
:100FE00092959F70963079F010F4925001C09A500B
:100FF000923068F4803F69F018F4883E40F409C0EC
:10100000843F29F406C0883E20F0813F11F080E043
:10101000089581E00895FC01808191810E94DB099F
:101020000E94F0070895CF93DF9300D000D01F9265
:10103000CDB7DEB70F900F900F900F900F90DF910C
:10104000CF910895CF93DF9300D000D000D0CDB7DB
:10105000DEB726960FB6F894DEBF0FBECDBFDF9188
:10106000CF910895089508950C9433080C94340892
:101070000E9436086093FA017093FB018093FC0193
:101080009093FD010C94D8070C9438080F931F938C
:101090000091FA011091FB012091FC013091FD01BA
:1010A000602B712B822B932B1F910F910C9438087E
:1010B0000F931F930091FA011091FB012091FC0105
:1010C0003091FD0160237123822393231F910F919F
:1010D0000C9438080F931F930091FA011091FB01B3
:1010E0002091FC013091FD01602771278227932711
:1010F0001F910F910C9438080C9433080E947C08BF
:101100006093F6017093F7018093F8019093F901D1
:101110000C94D80760E070E0CB010C947E080F932C
:101120001F9341E050E060E070E08A019B0104C041
:10113000000F111F221F331F8A95D2F7C901B80172
:101140001F910F910C947E080F931F9341E050E084
:1011500060E070E004C0440F551F661F771F8A953A
:10116000D2F78091F6019091F701A091F801B0912A
:10117000F9018A019B01082B192B2A2B3B2BC90152
:10118000B8011F910F910C947E080F931F9341E0BB
:1011900050E060E070E004C0440F551F661F771FE9
:1011A0008A95D2F740955095609570958091F6019B
:1011B0009091F701A091F801B091F9018A019B018A
:1011C000082319232A233B23C901B8011F910F913A
:1011D0000C947E080F931F9341E050E060E070E0B4
:1011E00004C0440F551F661F771F8A95D2F7809160
:1011F000F6019091F701A091F801B091F9018A01EF
:101200009B01082719272A273B27C901B8011F91ED
:101210000F910C947E080F931F930091F60110918B
:10122000F7012091F8013091F901602B712B822B8D
:10123000932B1F910F910C947E080F931F93009195
:10124000F6011091F7012091F8013091F901602326
:101250007123822393231F910F910C947E080F9387
:101260001F930091F6011091F7012091F801309140
:10127000F90160277127822793271F910F910C9402
:101280007E08089520E1929F800D1124E82FE695B5
:10129000E695E695877051E001C0550F8A95EAF70B
:1012A00085E0E89FF0011124EC53FE4F20E030E090
:1012B00070E04081CB01022E02C0969587950A947A
:1012C000E2F78170819584278523842781932F5F9E
:1012D0003F4F2530310569F7089520E1929F800D39
:1012E0001124682F669566956695982F977085E00E
:1012F000689FB001112440E050E080E0FB01E40F62
:10130000F51FEC53FE4F208130E0092E02C03695C8
:1013100027950A94E2F721703327042E01C0220F8B
:101320000A94EAF7822B4F5F5F4F4530510531F742
:101330000895BF92CF92DF92EF92FF920F931F9387
:10134000CF93DF938C01C090F601D090F701E0902D
:10135000F801F090F9018091FA019091FB01A091C0
:10136000FC01B091FD01C82AD92AEA2AFB2ACFE163
:10137000D0E0D701C6010C2E04C0B695A79597956D
:1013800087950A94D2F780FD04C0219790F7B12C7D
:1013900007C0BC2EB8018C2F0E94DC100197A9F366
:1013A0008B2DDF91CF911F910F91FF90EF90DF90E8
:1013B000CF90BF900895CF93DF93EC010E949909DD
:1013C000BE010E94DC10DF91CF9108951F93CF934F
:1013D000DF93EB019091C301992321F0CB010E948F
:1013E000DB0913C0882349F0CB010E949909182F0B
:1013F000682FCE010E94420904C0CB010E946D09F2
:10140000182FBE01812F0E94DC10DF91CF911F9118
:1014100008951F93CF93DF93C091FE0116E0809152
:10142000FF01C81799F0D0E01C9FF0011D9FF00D3F
:101430001124E050FE4F408151816281738184818B
:1014400095810E9422082196C770E9CFDF91CF9144
:101450001F91089540913002509131026091320203
:101460007091330280913402909135020C942208DD
:10147000EF92FF920F931F93CF93DF9380913502EA
:1014800082958F7009F065C080913202882309F43B
:1014900060C08091FE01F090FF0110913002009138
:1014A0003102609133027091340291E01F3F09F0E4
:1014B00090E0C0910001D0910101292F96E0E92E22
:1014C0008F1509F446C06115710521F00F3F21F019
:1014D00030E003C031E001C0322F90E030FD36C073
:1014E000E89EF001E99EF00D1124DF01A050BE4FEF
:1014F00011963C911197301329C03C91311326C0AD
:1015000012963C911297311121C013964D915C9126
:101510001497461B570B4C175D07C0F4809135029A
:101520008F70806180933502EB5FFD4F80818F70FB
:101530008061808380E392E00E94A407DF91CF91D5
:101540001F910F91FF90EF900C94090A01968770FC
:10155000B7CFDF91CF911F910F91FF90EF9008953A
:101560009F92AF92BF92CF92DF92EF92FF920F9332
:101570001F93CF93DF93CDB7DEB761970FB6F89483
:10158000DEBF0FBECDBF8C0185E0F801DE011D96E8
:1015900001900D928A95E1F7D8011296EC90909106
:1015A0003002E09131022091330230913402211552
:1015B000310531F0EF3F31F481E09F3F19F403C072
:1015C00081E001C080E0B82FB1709B2E80FD47C143
:1015D000D8014C9111965C9111971396AD90BC90E7
:1015E000149780E3C82E82E0D82EF0903202B50125
:1015F000621B730B2091000130910101FF2009F45F
:10160000D9C0809135026217730708F095C0282F62
:10161000207F09F052C05E1313C0491311C0FE2C85
:10162000E1100EC08F708061809335020E942A0AFB
:10163000C6010E94A40780913502F80185834DC13F
:10164000AB2831F05F3F31F481E04F3F19F403C024
:1016500081E001C080E080FD03C081E08E2502C0F2
:1016600080E090E0F82FF170FF2E80FF1CC0809189
:10167000FE012091FF0136E0821709F40BC190E0D2
:10168000389FF001399FF00D1124E050FE4F618129
:10169000561306C06081461303C06281E61203C080
:1016A00001968770E9CFFE2CEE2009F416C18091D7
:1016B000350281608093350254C05E1306C0491321
:1016C00004C0E11002C0F80199C0C8010E940B08D3
:1016D000882361F1EE2051F120913502822F82950D
:1016E0008F7090E0029774F08091300290913102F7
:1016F00098878F831986BB86AA862C87CE0107968A
:101700000E94A40786E0F801A0E3B2E001900D92E8
:101710008A95E1F70E94380A0E942A0A0AC05E17D9
:1017200011F1C8010E940B0881112CC0C8010E9450
:10173000A407FF24F394D1C0282F207F81F77A2DAE
:10174000B98AA88A6E2D89890E94130880E392E0E5
:101750000E94A40786E0D6011D928A95E9F70E94AF
:101760002A0AF12CBAC04913DCCFE110DACFF80114
:101770008583C8010E94A40786E0D6011D928A9540
:10178000E9F7ABC0EE2091F220913502822F8295CD
:101790008F7090E002970CF4B5CF80913002909159
:1017A00031029A8389831B82BD82AC822E83CE0153
:1017B0000196A6CF6217730708F044C0FE2CEE20F6
:1017C00009F4B4CF5E1330C049132EC02091350206
:1017D00020FD21C0822F82958F70482F50E0411547
:1017E0005105C9F0F80125834F30510541F08F5F55
:1017F000982F9295907F822F8F70892B8583C801B7
:101800000E94A40786E0F801A0E3B2E001900D92E7
:101810008A95E1F73CC086E0F801A0E3B2E00190D0
:101820000D928A95E1F759C0C8010E940B088111F9
:1018300069CF80913502816080933502C8010E9492
:10184000A4074BC07A2DB98AA88A6E2D89890E9477
:10185000130886E0D6011D928A95E9F718C0EE209C
:1018600009F464CFC8010E940B08F82E882309F4FC
:101870005DCF86E0F801A0E3B2E001900D928A9579
:10188000E1F780E392E00E9431040E94380A0E944E
:101890002A0A23C04D875E878D859E850E94DB09BD
:1018A000292F22952F70223028F49F7039F0811152
:1018B00005C00BC0243028F49F7049F4805E883046
:1018C00020F0C8010E94A4079F2CF92C06C0D80163
:1018D00015969C91907F91F7F8CF8F2D61960FB65A
:1018E000F894DEBF0FBECDBFDF91CF911F910F9156
:1018F000FF90EF90DF90CF90BF90AF909F900895B2
:101900001F93CF93DF93CDB7DEB72C970FB6F89424
:10191000DEBF0FBECDBF4F83588769877A878B871D
:101920009C87CE0107960E94B00A8823D1F09F8140
:1019300088852A853B85232B31F08F3F31F481E068
:101940009F3F19F403C081E001C080E080FD47C0E3
:101950004F81588569857A858B859C850E942208F0
:101960003EC086E0FE013796DE01119601900D9291
:101970008A95E1F7FF81E8856A857B8561157105A8
:1019800031F0EF3F31F481E0FF3F19F403C081E013
:1019900001C080E080FD23C02091FF0130E0C9013B
:1019A0000196877099274091FE0150E084179507B2
:1019B000F1F1F983EA837D836C8396E0929FD001F5
:1019C000939FB00D1124A050BE4FFE01319601909F
:1019D0000D929A95E1F78093FF010E94090A16E0A3
:1019E0008091FE019091FF01891771F1189FC0014C
:1019F000112480509E4F0E94B00A882329F1E09163
:101A0000FE011E9FF0011124E050FE4F40815181E4
:101A100062817381848195810E9422088091FE01F8
:101A200090E00196877099278093FE01D9CF0E949C
:101A3000EC071092FF011092FE01E0E3F2E086E075
:101A4000DF011D928A95E9F72C960FB6F894DEBF58
:101A50000FBECDBFDF91CF911F91089580915602A7
:101A6000859585958595089580915602877008958E
:101A700090915602977081E009F480E0089580917A
:101A80007902089590917902892B809379020895C3
:101A9000809590917902892380937902089510921C
:101AA0007902089590917802892B809378020895A5
:101AB00080959091780289238093780208951092FE
:101AC0007802089580915702089508950C94650D49
:101AD0000C94660D9091CE0292FD08C09091570231
:101AE000981721F0809357020C94680D0895809107
:101AF0005702882329F01092570280E00C94680D59
:101B00000895CF93DF93E0910201F091030180915A
:101B100079028083E0910201F0910301908180912C
:101B20007802892B808380915702882381F0E0918D
:101B30000201F09103019081892B80838091020141
:101B4000909103010E94121F81110E94770DC09194
:101B50000201D091030140E250E066E372E0CE0161
:101B60000E943E28892B69F080E2FE01A6E3B2E0E4
:101B700001900D928A95E1F7CE01DF91CF910C94FF
:101B8000CC1EDF91CF9108950C94650D9091CE02FB
:101B900092FD10C098E0899F90011124262B20937C
:101BA00056020E94A40880915602859585958595D8
:101BB0000C94C40D0C94A4081092560280E00C946E
:101BC000C40D209156028095822380935602982F4F
:101BD000977099F430E0482F082E000C550B24170D
:101BE000350759F09091CE0292FD07C085958595F5
:101BF00085950E94C5080C94DC0D08959091CE0245
:101C000092FB222720F9281769F080FB92F9909324
:101C1000CE028091CD029091CE020E944C0E82E0C5
:101C20000C94E10D08958091CE0282FB882780F903
:101C300091E089270C94FE0D81E00C94FE0D80E06C
:101C40000C94FE0D6FEF7FEF80E090E00C947D2808
:101C500080E090E00E94592821E0893E9E4F09F0E3
:101C600020E0822F089582E090E00C944B2883E0DE
:101C700090E00C944B28CF9384E090E00E944B2896
:101C8000C82F82E290E00E944B282C2F30E0A9015F
:101C9000582BCA01CF910895CF93C92F682F84E0A4
:101CA00090E00E945F286C2F82E290E0CF910C942C
:101CB0005F28AB01BC018FE090E00C947128AB0170
:101CC000BC0183E190E00C94712860E070E0CB01EE
:101CD0000C945F0E60E070E0CB010E94590E0C94F2
:101CE000650E69EE7EEF80E090E00E947D2860E066
:101CF00082E090E00E945F2860E083E090E00E9434
:101D00005F281092FA011092FB011092FC011092D0
:101D1000FD0160E084E090E00E945F2860E082E2E4
:101D200090E00E945F2860E085E090E00E945F28DC
:101D300060E086E090E00E945F286FEF87E090E02F
:101D40000E945F2840E050E0BA0188E090E00E94E5
:101D5000712860E08DE090E00E945F2840E050E054
:101D6000BA0188E190E00E94712860E087E190E08C
:101D70000E945F2840E050E0BA018CE190E00E94B0
:101D8000712860E070E080E290E00E947D2840E0F1
:101D900050E0BA0188E190E00E9471280C946A0E2C
:101DA0000C94710E682F8EE090E00C945F280E94D6
:101DB0007820609388027093890280938A029093BE
:101DC0008B026093840270938502809386029093C5
:101DD0008702089585B7806885BF85B7806885BF0D
:101DE000089581E008950C94F10E08950C94F50E79
:101DF0000C94F50E0C94F80E0C94F50E0C94FC0E4D
:101E00000C94F50E0E94EA0E88EB91E10E94B61E3A
:101E10000E94000F0C94FE0E0E94F60E0C94F50E1C
:101E20000E94D2110E94C9030C943D1C0E946320A1
:101E30000E94B7120E94100F0E94761A0E94B518D5
:101E40000C94FA0E5F926F927F928F929F92AF9254
:101E5000BF92CF92DF92EF92FF920F931F93CF9397
:101E6000DF93CDB7DEB72A970FB6F894DEBF0FBE6B
:101E7000CDBF0E94CC12C82E81110E94D70E3AE726
:101E8000832E32E0932E00E010E0502E802F0E942F
:101E9000F6115C01F401619071904F01682679267A
:101EA00061147104B1F40F5F1F4F0530110569F71C
:101EB0008FEF89838A831B820E946C208160782F38
:101EC0009D838C8349815A816B818D810E94E703B8
:101ED0003AC080918C0281FD0E94FF11D12CEE242A
:101EE000E394F12CC3018E219F21892B29F10E94BB
:101EF000F30E8823A9F0DE825F82AE20BF2081E04E
:101F0000AB2809F480E088870E946C208160782FDC
:101F10009A8789874E815F8168858A850E94E70359
:101F2000000F111FF801E658FD4F80819181E826CE
:101F3000F926F182E08207C0D394EE0CFF1CF0E199
:101F4000DF12D0CFB0CF81E0C11001C080E02A966F
:101F50000FB6F894DEBF0FBECDBFDF91CF911F91BA
:101F60000F91FF90EF90DF90CF90BF90AF909F9038
:101F70008F907F906F905F9008950E94220F0E9433
:101F8000E8180E943C1C0C94DC03CF93DF930E9462
:101F9000E110EC01811522E59207E8F5811531E5A4
:101FA000930708F0B6C0883E910528F5803E91055C
:101FB00008F0E9C0883A910570F4853A910508F077
:101FC0007AC08130910509F473C008F4D9C0049730
:101FD00008F0D9C0D5C08F3B910508F0D1C0C85AD0
:101FE000D0E0CC0FDD1FCB5ADE4F0990D881C02D39
:101FF000CE019464C9C0811540E5940708F069C01A
:10200000811550E4950708F060C09A9581159F41AD
:1020100008F4B9C0B5C0811536E5930728F58115D8
:1020200045E5940708F092C0811554E5950708F03E
:1020300087C0AC0143705527282F26952695C115DA
:10204000D34508F06CC081E090E002C0880F991F72
:102050004A95E2F740E2249F90011124EC01C22B43
:10206000D32BCE019C6890C081152AE5920780F49D
:10207000811539E5930708F072C0811548E594078A
:1020800008F47EC0D82FCC27CE01806F906A7CC028
:1020900090568115904208F073C08D2F8F710E9469
:1020A0007511DD27D0628F71AE01582BCA016CC04B
:1020B00081E090E069C0C55AD0E0CD57DE4F8881FD
:1020C000C82FD0E0CE0190645FC0DF70CE01906A6F
:1020D0005BC074E0969587957A95E1F7282F237079
:1020E0003C2F337081E090E002C0880F991F3A9531
:1020F000E2F79C68AC01522B9A019C2F9F70969539
:10210000969550E2959FE0011124C9018C2B9D2BDF
:102110003BC0D82FCC27CE01816F906A35C081E0BB
:1021200090E002C0880F991F4A95E2F750E2259F80
:1021300090011124EC01C22BD32BCE019A6824C04C
:10214000D82FCC27CE01846F906A1EC00E947511D3
:102150008F7190E0D82FCC27CE01906215C08F7080
:102160000E94751194E0D695C7959A95E1F7CF70C6
:10217000D0E0DC2FCC27D0699E01282BC90104C0F8
:1021800080E090E001C0CE01DF91CF910895E72F6C
:10219000F0E095E0899FE00DF11D112484E0EE0F41
:1021A000FF1F8A95E1F7E60FF11DEE0FFF1FE852C2
:1021B000FF4F8591949108950E94C7100E94C50F0A
:1021C00008958238910569F1B0F48133910509F4DD
:1021D0006DC048F48932910509F463C08A329105D3
:1021E00009F469C008958533910509F455C0893310
:1021F0009105B9F00895833E910569F138F4803E68
:102200009105B1F0823E910509F10895863E910550
:10221000A9F1873E9105B9F1843E910509F064C0AA
:1022200023C02091CD0220FD4FC021FD4DC0089557
:102230008091CD0280FD44C08091CE0280FF44C0D9
:102240008091CD0284FD42C083EE4DC08091CD02CD
:1022500082FF38C0F5CF8091CD0282FD33C08091DE
:10226000CE0280FD31C0ECCF8091CE0281FF32C022
:102270008091CD0284FD2AC087EE35C08091CD02C9
:1022800083FF26C0F5CF8091CD0283FD21C08091D0
:10229000CE0281FD1FC0ECCF8091CD0285FD1CC018
:1022A0001DC08091CD0285FD19C016C08091CD0260
:1022B00086FD16C017C08091CD0286FD13C010C0E8
:1022C00089E311C082EE0FC080EE0DC080E00BC02C
:1022D00086EE09C084EE07C089E205C085E303C02D
:1022E0008AE201C081E390E008959091CD0292FFCF
:1022F0000DC0282F2871283019F4877F846006C00C
:10230000282F2471243011F48B7F886093FF0DC037
:10231000282F2871283119F4877E846106C0282F60
:102320002471243111F48B7E88612091CE0220FF2C
:102330000DC0382F3871383019F4877F816006C09E
:10234000382F3171313011F48E7F886021FF0DC03C
:10235000282F2871283119F4877E816106C0282F23
:102360002171213111F48E7E886194FD877E08955C
:1023700080E008950C94220E0E94CC128FE39CE919
:102380000197F1F700C000000E94CC1280E00E948B
:10239000F61180FF04C00E94BA110C94B920089570
:1023A0000C94BC110E94280E811102C00E94D00E14
:1023B0000E94330E80938C020E943B0E9093CE02BB
:1023C0008093CD020E94D0110E94370E682F70E0DA
:1023D00080E090E00E9444086091F6017091F7015E
:1023E0008091F8019091F9010C947C08E82FF0E0BD
:1023F000EE0FFF1FE752FD4F8081918108950895F0
:1024000080EA8A95F1F7089500C008950C940012AF
:1024100008950C9408120C9409120C9408120C9450
:102420000D12F894E82FE295EF70F0E031A1282F1B
:102430002F7081E090E001C0880F2A95EAF7982F6D
:102440009095932391A392A1892B82A378940895C8
:102450000F931F93CF93DF93C6E9D1E089918F3F0C
:1024600011F00E94111281E0CB39D807B9F7C6E804
:10247000D1E006E911E089918F3F11F00E9411121D
:102480000C171D07C1F7DF91CF911F910F91089590
:10249000BF92CF92DF92EF92FF920F931F93CF9351
:1024A000DF938C01C62FD0E0CE018A569E4F6C017F
:1024B000FC0190819F3F09F450C0B62EF894E92F9B
:1024C000E295EF70F0E081A19F7021E030E001C063
:1024D000220F9A95EAF7822B81A382A120952823C7
:1024E00022A378940E940412E6E8F1E046E951E064
:1024F00021E030E0E12CF12C61916F3F89F0A62FB3
:10250000A295AF70B0E090968C9190E06F7002C091
:10251000959587956A95E2F780FD02C0C90102C0D2
:1025200080E090E0E82AF92A220F331F4E175F0758
:1025300019F7F60180818F3F11F00E94111261E0BE
:10254000E114F10409F460E08B2D0E940612CC0F17
:10255000DD1FC00FD11FF982E882DF91CF911F915B
:102560000F91FF90EF90DF90CF90BF9008950E9461
:1025700028128AE0E9EDF2E0DF01982F1D929A958A
:10258000E9F7EFECF2E0DF011D928A95E9F785E0CB
:102590000E9417130C943603FF920F931F93CF934F
:1025A000DF93CDB7DEB72A970FB6F894DEBF0FBE24
:1025B000CDBF8E010F5F1F4F8AE0F80111928A95FF
:1025C000E9F7F12C6F2DC8010E944812F394F5E051
:1025D000FF12F8CF4AE050E0B8018FEC92E00E9481
:1025E0003E28FF24F394009709F4F12C892B41F045
:1025F0008AE0F801AFECB2E001900D928A95E1F724
:102600002F2D45E069ED72E08FEC92E00E941813E7
:102610000E9438038F2D2A960FB6F894DEBF0FBEA6
:10262000CDBFDF91CF911F910F91FF900895089535
:10263000FF920F931F93CF93DF93F82E092F162F3E
:10264000D72FC42F222349F081E080938F020E946C
:102650006C2090938E0280938D0280918F0288234C
:10266000D9F080918D0290918E020E94842005976E
:1026700098F0EF2DF02FA12FBD2F80E090E04C2F90
:1026800050E08417950734F4219131912D933D93B7
:102690000196F7CF10928F02DF91CF911F910F918A
:1026A000FF9008950E9466220E94160F0C947222D9
:1026B0000E9476220E94BD0F0C9490220E940A2054
:1026C0000E944D220E94020F0E9452130E94581332
:1026D0000E940C0FFBCFEF92FF920F931F93CF93AB
:1026E000DF938B01682F11110AC0442329F0E82FD2
:1026F000F0E0E15DFC4F6491762F862F75C0212FAD
:1027000030E0E82FF0E0442321F0E15DFC4FE4915C
:10271000F0E046E0049FC0011124CFEFD0E0BE01FD
:102720000E94B0274BEA4603C001479F900D112439
:10273000800F911D800F911D982F990F890FAE0169
:10274000421B530B4E9FD0014F9FB00D5E9FB00DAB
:1027500011249B2F189FA0011124452F55278E016E
:10276000041B150B0E9FA0010F9F500D1E9F500DB7
:1027700011247E01E81AF108E29E8001E39E100D0B
:10278000F29E100D1124212F3327C21BD30BCE9F95
:102790009001CF9F300DDE9F300D11246230710506
:1027A000A9F048F46115710569F061307105C9F44B
:1027B0008B2F752F0DC06430710581F058F0663095
:1027C000710579F47E2F8B2F932F0DC0832F7B2FD4
:1027D0009E2F09C08E2F7B2F952F05C08E2F732F14
:1027E00002C07E2F852F692FDF91CF911F910F910E
:1027F000FF90EF90089541E00E946B1308950895B3
:102800000E94FB130895CF93DF93762FE901682F81
:10281000842F0E940014798368838A83DF91CF918B
:1028200008958091E302282F269530E02115310587
:1028300019F48170826005C02532310524F0817061
:1028400088648093E302089588E090E00C94532814
:10285000CF92DF92EF92FF926B017C010E941114E4
:10286000B701A60188E090E0FF90EF90DF90CF9055
:102870000C947128E3EEF2E083E0808311828FEF05
:1028800082838383148260817181828193810C941D
:1028900028148091E30280FF02C08695089580E0AD
:1028A00008959091E702933018F49F5F9093E702A8
:1028B000882351F06091E3027091E4028091E50277
:1028C0009091E6020C942814089581E00C94511420
:1028D0009091E702992319F091509093E702882391
:1028E00051F06091E3027091E4028091E5029091D1
:1028F000E6020C942814089581E00C94681470E0AA
:102900000C944D1C609108018091E30280FF0AC085
:102910008091070123E0829FC001112488519D4FBF
:102920000C947F148091090190910A01891780F716
:10293000E82FF0E09F01220F331FE20FF31FE85151
:10294000FD4F1182108212828F5FF0CF9091E302CF
:1029500090FF16C09091090120910A01921770F41E
:10296000E92FF0E0DF01AA0FBB1FEA0FFB1FE851C0
:10297000FD4F8183608342839F5FF0CF0C9482146C
:102980000895CF93DF9300D01F92CDB7DEB790911B
:10299000E30290FF0AC09E012F5F3F4F0E94031485
:1029A0004B8169818A810E94A6140F900F900F902D
:1029B000DF91CF910895CF93DF93EC01EC81F0E0AC
:1029C000E65DFD4F4491E3EEF2E0628181810E9479
:1029D000C1148C818F5F8C83DF91CF910895CF9349
:1029E000DF93EC01E3EEF2E0438162818C810E948F
:1029F000C1148C818F5F8C83DF91CF9108950F93E9
:102A00001F93CF93DF9300D01F92CDB7DEB78C0119
:102A10008091900281110AC09E012F5F3F4F4FEFBE
:102A20006FEF0E9403148A8180939002F8018481E1
:102A3000813051F028F0823061F4409190020AC058
:102A40008091900240E007C06091900240E080E0F9
:102A500003C040E080E060E00E94A614F801848199
:102A600090E0019663E070E00E94C42784830F9099
:102A70000F900F90DF91CF911F910F910895AF921A
:102A8000BF92CF92DF92EF92FF920F931F93CF935B
:102A9000DF9300D01F92CDB7DEB7182FF62E042F8C
:102AA000E22E9091E30290FF6DC0E92FE695AE2FE4
:102AB000B0E0A556BE4F8C9180939A029E7F9230D3
:102AC00061F49E012F5F3F4F812F0E9403144B81C1
:102AD00069818A810E94A61443C0823019F4009152
:102AE000E6023EC0863019F41091E40239C0893004
:102AF000D9F38931A9F5E9518E2F8170D82EE69549
:102B0000F0E0E65DFC4FA590B490C12CBB24609131
:102B10000B01C61618F52C2D30E0A29EC001A39E15
:102B2000900DB29E900D112470E00E94B027812F6D
:102B3000D11002C0860F01C0861B90910901290F98
:102B4000311DA901440F551F240F351F28513D4F3A
:102B5000402F6F2D0E940314C394D9CF0E9482147A
:102B60001093E402F092E5020093E602EE2051F0A9
:102B70006091E3027091E4028091E5029091E60297
:102B80000E9428140F900F900F90DF91CF911F910A
:102B90000F91FF90EF90DF90CF90BF90AF9008958E
:102BA000E3EEF2E09181282F4381628180E1890F79
:102BB0000C943F1581E00C94D015E3EEF2E0918186
:102BC000282F4381628180EF890F0C943F1581E0AB
:102BD0000C94DD15E3EEF2E0628120E1620F08F46F
:102BE0006FEF282F438181810C943F1581E00C9475
:102BF000EA15E3EEF2E0628120E1621B08F460E096
:102C0000282F438181810C943F1581E00C94F915A4
:102C1000E3EEF2E0438120E1420F08F44FEF282F6A
:102C2000628181810C943F1581E00C940816E3EEDB
:102C3000F2E0438120E1421B08F440E0282F62814A
:102C400081810C943F1581E00C94171620E00C94C0
:102C50003F15FF920F931F93CF93DF93EC01F12C5D
:102C60000FEF10E060910B01F616F0F4809109016E
:102C70002F2D30E0280F311DC901880F991F280F13
:102C8000391F28513D4F70E0C8010E94C427962F7C
:102C90008C814091E6026091E502F99E800D11243D
:102CA0000E940314F394DECF0E9482149A818C81D7
:102CB00090FF02C08F5F01C081508C83DF91CF9164
:102CC0001F910F91FF900895BF92CF92DF92EF92E4
:102CD000FF920F931F93CF93DF93FC01828180FFBC
:102CE00002C00FEF01C001E010E080910B01181746
:102CF00008F040C080910901C12ED12CE601C80F17
:102D0000D11DCE01880F991FC80FD91FC851DD4FA3
:102D1000198218821A8234E0E32EF12CB12C8091B2
:102D200092028B0D813114F08F7005C087FF03C0B4
:102D300090910B01890F082E000C990BC816D9062B
:102D400091F48091E6028E9DA0018F9D500D11247B
:102D500055954795559547959E016091E50280915F
:102D6000E4020E940314B00EF1E0EF1AF108B9F684
:102D70001F5FBBCF0E94821480919202013031F418
:102D8000811102C080910B01815007C090E0019633
:102D900060910B0170E00E94C42780939202DF9142
:102DA000CF911F910F91FF90EF90DF90CF90BF9048
:102DB0000895CF938091090190910A01891770F4C9
:102DC000E82FF0E09F01220F331FE20FF31FE851BD
:102DD000FD4F1182108212828F5FF0CFC0E06091B0
:102DE0000B01C617C0F5EC2FF0E070E0CF010E9498
:102DF000C42720910901820F20919102022E000C1C
:102E0000330B90E0E217F307CCF020910601022E7D
:102E1000000C330B2E173F078CF09C01220F331F41
:102E2000820F931F9C0128513D4F4091E602609113
:102E3000E5028091E4020E9403140BC0FC01EE0F36
:102E4000FF1F8E0F9F1FFC01E851FD4F1182108262
:102E50001282CF5FC4CF0E9482142091050180911D
:102E60009102820F8093910290910601920F9093AC
:102E7000060119165CF4082E000C990B40910B0109
:102E800050E041505109841795071CF0219520937B
:102E90000501CF9108958F929F92AF92BF92CF92EA
:102EA000DF92EF92FF920F931F93CF93DF938C01EA
:102EB000FC014481C42FD0E09E01DE010E9408285D
:102EC0009B01AC010E941E286B017C01E0E2F0E056
:102ED000EC1BFD0BA5E5B0E09B01AC010E941E2898
:102EE0004B015C019F01DF010E9400289B01AC01A6
:102EF0000E9429289B01AC012C0D3D1D4E1D5F1D1C
:102F0000C501B4010E94D827C22FD22F2A3228F43B
:102F1000F3E02F9F900111240DC025E530E02C1B1C
:102F20003109C901880F991F280F391F37FF02C0C7
:102F30002F5F3F4F35952795C22FC095F12C85E522
:102F4000E82EED1A80910B01F816C8F4F1FC02C0CE
:102F50008E2D01C08D2F909109012F2D30E0290F6A
:102F6000311DA901440F551F240F351F28513D4F16
:102F70004C2F6091E5020E940314F394E3CF0E946A
:102F80008214F8018481811102C091E003C0803273
:102F900019F49FEF9093040190910401890FF801B7
:102FA0008483DF91CF911F910F91FF90EF90DF907D
:102FB000CF90BF90AF909F908F9008950F931F93E5
:102FC000CF93DF93EC0100E010E080910B01282FFC
:102FD00030E00217130724F5909109019801290F99
:102FE000311DA901440F551F240F351F28513D4F96
:102FF000869590E04C81081719071CF4442331F0A2
:1030000002C0411103C04091E60201C040E060915E
:10301000E5028091E4020E9403140F5F1F4FD5CF99
:103020000E9482148C8190E00196817099278C8394
:10303000DF91CF911F910F910895E3EEF2E080812F
:103040008E7F808360817181828193810E942814A8
:1030500010929B022FEF80E792E021508040904039
:10306000E1F700C000000C9482146091E3026695C1
:1030700070E04BE050E08CE091E00E943128892B19
:1030800019F481E080939B020E946C20909394023B
:103090008093930208959091E30290FF35C0917060
:1030A000811102C0926006C0853210F0986402C09F
:1030B000880F982B9093E302662351F06091E3020E
:1030C0007091E4028091E5029091E6020E9428143A
:1030D0006091E302669570E04BE050E08CE091E097
:1030E0000E943128892B19F010929B0202C00E9485
:1030F000351881E0809396024091E6026091E502E6
:103100008091E4020C9426160895682F9091E302B2
:10311000969581E0890F853208F081E00C944B1878
:1031200081E00C948518682F9091E30296958FEFBB
:10313000890F09F484E20C944B1881E00C949318E5
:1031400061E00C944B18E3EEF2E0808181608083B3
:1031500086950C94A0188091E30280FD0C941D18B4
:103160000C94A31860E00C944B1880919902811183
:103170002EC00E94280E811104C00E94D00E0E9411
:103180003A140E9424146093E3027093E402809343
:10319000E5029093E6026E7F61F40E943A140E9469
:1031A00024146093E3027093E4028093E502909309
:1031B000E6020E94111410929B028091E30280FFAC
:1031C00003C086950E94B21881E080939902089509
:1031D0000F931F93CF93DF9380919B02882309F471
:1031E00085C080919A02E091E302E695E81BE093A6
:1031F0009502823049F4F0E0EA5DFD4FE491CE2F74
:10320000D0E00BED14E149C0863049F4F0E0ED5D0B
:10321000FD4FE491CE2FD0E00FEE14E13EC0893097
:1032200051F4E695F0E0E05EFD4FE491CE2FD0E062
:1032300009E216E132C08F3051F4E695F0E0E35E2A
:10324000FD4FE491CE2FD0E004E616E126C0853193
:1032500049F4F0E0E65EFD4FE491CE2FD0E009EDB9
:1032600016E11BC0883181F0833239F4E8E1F2E0E5
:10327000C591D4910FEF14E110C0843251F4C4EF22
:10328000D1E00EED17E109C0C8E2D0E00BE417E190
:1032900004C0C0EDD7E00FEF13E1809196028823C0
:1032A00061F0109296020E946C2090939402809399
:1032B000930210929802109297020E946C20E09163
:1032C0009302F09194028E1B9F0B8F3F9F4770F4E7
:1032D000EC0FFD1FF0939402E093930283E992E0D8
:1032E000F801DF91CF911F910F910994DF91CF9158
:1032F0001F910F910895882311F0FA0101C0FB017D
:103300000994CF93DF93C82FD62F0E9449148C17AE
:1033100040F00E9449148D1720F4DF91CF910C9456
:1033200090188C2FDF91CF910C94A0181F93CF93FE
:10333000DF93FB0112811111C3C0EC010E943F0D0C
:103340008272CD3CFCE5DF0709F49AC0A8F5C73CC2
:10335000ECE5DE0709F476C0A8F4C43C9CE5D90787
:1033600009F45FC028F4C33CDC4509F457C054C0DD
:10337000C53C9CE5D90709F459C0C63CDC4509F4B5
:103380005CC04AC0CA3CFCE5DF0709F46AC050F4DF
:10339000C83CECE5DE0709F45AC0C93CDC4509F439
:1033A0005BC03AC0CB3C9CE5D90709F45FC0CC3C7C
:1033B000DC4509F460C030C0C23DFCE5DF0709F41C
:1033C0006FC088F4CF3C9CE5D90709F460C008F4CD
:1033D0005CC0C03DFCE5DF0709F45CC0C13DDC45D5
:1033E00009F45BC019C0C53D9CE5D90709F460C06C
:1033F00050F4C33DFCE5DF0709F455C0C43DDC458E
:1034000009F454C009C0C63D9CE5D90709F455C06C
:10341000CE35DD4509F454C011E052C00E94AB180E
:103420004FC04DE958E160E978E104C040E958E156
:103430006DE978E10E947B1943C047EE55E16AEDE2
:1034400075E1F8CF4AED55E167EE75E1F3CF45E060
:1034500056E166EF75E1EECF46EF55E165E076E1C6
:10346000E9CF43E256E164E176E1E4CF44E156E19D
:1034700063E276E1DFCF4CE754E165E674E1DACF51
:1034800045E654E16CE774E1D5CF81E017C065E013
:1034900082E010C068E086E00DC06EE089E00AC0FE
:1034A00064E18FE007C067E185E104C088E106C000
:1034B00062E289E10E94811903C083E20E94A018A0
:1034C000812FDF91CF911F91089586E090E00C94B9
:1034D0004B28682F86E090E00C945F2880911803B9
:1034E00084708961809318030C94691A0E94280ED5
:1034F000811104C00E94D00E0E946E1A0E94651AAB
:1035000080931803282F26952695269530E02430A1
:10351000310524F087708861809318038091180327
:1035200080FF04C086958695869501C080E00C9446
:10353000871B20911803822F869586958695482FA4
:1035400050E04330510554F48F5F982F990F990F35
:10355000990F822F8770892B80931803809118030D
:103560008160809318030E94691A809118038695E0
:10357000869586950C94871B80911803982F9695B5
:1035800096959695A1F0915E990F990F990F877076
:10359000892B80931803887F91E009F490E0809153
:1035A000180390FB80F9809318030E94691A809198
:1035B00018038695869586950C94871B8091180331
:1035C00080FD13C0816080931803813019F489E075
:1035D00080931803809118030E94691A8091180340
:1035E0008695869586950C94871B0895809118037F
:1035F00080FF08C08E7F809318030E94691A80E0C4
:103600000C94871B08958091180380FD0C94F61A82
:103610000C94DE1A90911803892F869586958695CD
:103620008F5F8F719770843038F4880F880F880F00
:10363000892B8093180302C090931803809118037C
:10364000887F91E009F490E08091180390FB80F965
:10365000809318030E94691A8091180386958695B5
:1036600086950C94871B843008F083E090911803B2
:103670009770282F220F220F220F922B909318035E
:10368000987F21E009F420E09091180320FB90F945
:10369000909318030C94871B0E94331B809118038E
:1036A0000C94691A9C01FB018281882349F12E3B0D
:1036B000FCE53F07C9F040F42C3BECE53E0769F020
:1036C0002D3B3C4561F00895203C9CE5390791F085
:1036D00070F0213C3C4589F0089583E001C080E012
:1036E0000E944C1B80E008950E94BC1AFBCF0E94F0
:1036F000991AF8CF0E94031BF5CF0E940A1BF2CF44
:1037000081E00895279A2F9808952F9808958F9211
:103710009F92AF92BF92CF92DF92EF92FF920F9360
:103720001F93CF93DF93C82F843050F4811109C0C9
:1037300080918000877F809380000E94851B06C057
:10374000C3E080918000886080938000A091860013
:10375000B09187002C2F30E00E94082823E030E051
:1037600040E050E00E94D8270027122F232F342F4B
:10377000012F122F232F33278091860090918700ED
:103780006CE070E00E94B0276017710730F0C8014C
:1037900069E070E00E94B0275EC080918600909141
:1037A0008700E0908600F0908700E0918600F0911D
:1037B0008700C6E0D0E0BE010E94B027060F171FA9
:1037C000211D311D4801590185E0880C991CAA1C56
:1037D000BB1C8A95D1F7C701BE010E94B0276F01BB
:1037E000E12CF12CA7019601260F371F411D511D19
:1037F000C501B4010E94D82769017A01E0918600D1
:10380000F0918700CA01B9010E94A0279B01AC0179
:10381000DF010E941E289B01AC01C701B6010E9476
:10382000A027DC01CB012FE0B695A795979587954A
:103830002A95D1F7009186001091870020E030E0B2
:10384000081719072A073B0728F460918600709132
:103850008700CB01BC0170938D0060938C00DF91D9
:10386000CF911F910F91FF90EF90DF90CF90BF907D
:10387000AF909F908F90089508950E94821B8AE0D8
:103880008093800089E1809381008FEF9FEF909378
:103890008700809386000C94761A259A25B12F7D97
:1038A00035B130624FB7F894FC01CB01880F991FF6
:1038B000680F791F6E0F7F1FE617F70789F0819158
:1038C00098E035B9000000C087FF25B9880F0000D7
:1038D00000C000C000C025B900C09A9591F7ECCF98
:1038E0004FBF8FE594E00197F1F700C00000089505
:1038F000CF93DF93EC01FB018281882309F43CC163
:10390000C430FDE5DF0760F4CB3F9CE5D90788F4C0
:103910009E0122503C452431310508F02EC109C0DA
:10392000C236EDE5DE0729F0C63AFDE5DF0709F00E
:1039300024C10E943B0E9093CE028093CD02C131F0
:103940008CE5D80709F4C6C008F042C0C930ECE5E0
:10395000DE0709F49BC000F5C5308CE5D80709F4F3
:1039600085C078F4C330ECE5DE0709F478C008F0D0
:103970007AC0C230DC4509F0F5C08091CD0281608B
:10398000EFC0C7309CE5D90709F478C008F07AC0C9
:103990008091CD028061E4C0CD30FCE5DF0709F401
:1039A00087C058F4CB309CE5D90709F479C008F0FA
:1039B0007BC08091CD0288606FC0CF30FCE5DF070F
:1039C00009F480C008F082C08091CD02877FC8C012
:1039D000CE3F9CE5D90709F471C000F5C531FCE57F
:1039E000DF0709F485C068F4C3319CE5D90709F401
:1039F00075C008F095C00E94EC078091CD028F77CA
:103A0000AFC0CC3FFCE5DF07A9F108F054C0CB3FC5
:103A1000DC4509F0A7C08091CE0240C0C230EDE580
:103A2000DE0709F489C058F4C1158DE5D80709F4FB
:103A30005AC008F069C08091CE0282602FC0C236A1
:103A4000EDE5DE0709F47CC0C63AFDE5DF0709F4C1
:103A500081C0C330DD4509F085C080E06EC0809133
:103A6000CD0282607DC08091CD0216C08091CD02D2
:103A7000886076C08091CE0282604FC08091CD0276
:103A800080626EC08091CD0280646AC00E94EC07A3
:103A90008091CD02806864C0846062C081603DC056
:103AA0008091CD028E7F5CC08091CD028D7F58C009
:103AB0008091CD0216C08091CE0218C08091CE02B6
:103AC0008D7F2BC08091CD028F7E4AC08091CD0228
:103AD0008F7D46C08091CD028F7B42C08091CD0208
:103AE000877F8B7F3DC08091CE028D7F8E7F15C0FA
:103AF0008091CD0282FB222720F991E0922790FB52
:103B000082F990FB83F92CC08091CE02982F90957A
:103B100091708E7F892B90FB81F98093CE0222C019
:103B20000E94EC078091CD0287FB222720F991E0CB
:103B3000922790FB87F914C081E00E94D20E12C038
:103B40008091CD0284FB222720F991E0922790FBFF
:103B500084F906C08091CD02982F909590FB80F952
:103B60008093CD028091CD029091CE020E944C0EA6
:103B70000E94EC0780E001C081E0DF91CF910895C1
:103B8000CF93DF9386319C4541F5EB010E943F0DB9
:103B9000982F8A812091020130910301882379F0C6
:103BA0009A7A81E009F480E080939C02911102C02E
:103BB00069E201C065E3C9010E94A81F0AC08091A3
:103BC0009C02811102C069E201C065E3C9010E9443
:103BD000B31F0E94810D80E001C081E0DF91CF9191
:103BE00008950F931F93CF93DF93C42FD22FFC011F
:103BF00082818823C9F040939F020E946C20909399
:103C00009E0280939D0280E28C0F883008F057C09E
:103C1000C77081E001C0880FCA95EAF7DF91CF91A4
:103C20001F910F910C94580580919F02481330C04A
:103C300080919D0290919E020E948420883C910573
:103C400038F510E21D0FCD17B9F080E28C0F8830E7
:103C500040F4C77081E001C0880FCA95EAF70E945E
:103C60005F05183028F581E09D2F977001C0880FFF
:103C70009A95EAF70E945805802F0E944F05183048
:103C8000F0F4D77081E001C0880FDA95EAF70AC036
:103C900080E28C0F883098F4C77081E001C0880FF3
:103CA000CA95EAF7DF91CF911F910F910C945F05B0
:103CB000802FDF91CF911F910F910C944F05DF91D1
:103CC000CF911F910F9108950F939C01CB01243F39
:103CD0004CE5340731F188F4293DFCE53F07D9F084
:103CE0002A3D4CE5340779F1283D3C45A9F506E22B
:103CF00021EE41EE68ED7CE52BC0263FFCE53F0759
:103D0000E1F0A8F0273F3C4539F507E225EE46EE05
:103D100067EF7CE51DC007E225EE45EE69ED7CE529
:103D200017C006E221EE40EE64EF7CE511C007E229
:103D300025EE44EE65EF7CE50BC006E221EE42EE97
:103D400066EF7CE505C008E221E045EE6AED7CE522
:103D50000E94F11D80E008C0FC018281882319F0D7
:103D600010929F0201C081E00F9108959093C101CC
:103D70008093C00108959093A5028093A4020895B2
:103D8000E091A402F091A502309721F00190F0811A
:103D9000E02D099480E00895E091A402F091A5023D
:103DA000309799F020912301222359F02091CD02E0
:103DB00027FF07C0DC012C9111962C93119726E068
:103DC0002C930280F381E02D099408952091A202A2
:103DD0003091A3022817390771F09093A3028093C2
:103DE000A202E091A402F091A502309721F0068092
:103DF000F781E02D099408952091A0023091A1024D
:103E00002817390771F09093A1028093A002E091E6
:103E1000A402F091A502309721F00084F185E02DF5
:103E200009940895FC01329680912301882331F092
:103E30008091CD0287FF02C09EE101C096E080E044
:103E4000915028F021912223D9F38F5FF9CF089563
:103E5000662351F1209123012223E9F02091CD0224
:103E600027FF19C0462F4695469546954E31E0F4FA
:103E7000677021E030E002C0220F331F6A95E2F73D
:103E8000FC01E40FF11D828190E02823392381E0B9
:103E9000232B69F409C0FC01329608962191621720
:103EA00029F0E817F907D1F780E0089581E0089537
:103EB0009C01FC0132969FEF80E04191461789F00A
:103EC0009F3F19F4411101C0982F8F5F8630A9F7E9
:103ED0009F3F39F0F901E90FF11D97FDFA956283D3
:103EE000089508959C012A5F3F4FFC0142814613CB
:103EF00001C01282019682179307B9F70895262F01
:103F00002695269526952E3168F4FC01E20FF11DC9
:103F1000677021E030E001C0220F6A95EAF78281E4
:103F2000282B22830895262F2695269526952E3117
:103F300070F4FC01E20FF11D677021E030E001C078
:103F4000220F6A95EAF7209582812823228308951B
:103F500020912301222329F02091CD0227FD0C94EA
:103F60007F1F0C94581F20912301222329F02091B8
:103F7000CD0227FD0C94931F0C94721F20912301F6
:103F8000FC013296222331F08091CD0287FF02C0DE
:103F90008EE101C086E0DF011D928A95E9F7089560
:103FA00008950C94D01F83E08093A6020C94D11F37
:103FB000811102C081E001C082E08093A6020C94CE
:103FC000D11F0C94D81F81E08093A6020C94D11FBE
:103FD0000C94E31F08950C94EA1F0C94EB1F0C94AF
:103FE000EA1F0C94EA1F0C94EA1FCF930E94F11F62
:103FF0000E94CC120E94EF1FC0E08C2F0E94F6118D
:10400000892B29F4CF5FC530C1F780E001C081E082
:10401000CF91089508951F920F920FB60F92112419
:104020008F939F93AF93BF938091A702811113C089
:104030008091190390911A03A0911B03B0911C0366
:104040004196A11DB11D8093190390931A03A0936B
:104050001B03B0931C03BF91AF919F918F910F9061
:104060000FBE0F901F90189580912103843031F17D
:104070000E94AA031092A70220E488E190E00FB604
:10408000F894A895809360000FBE2093600083B7DA
:10409000817F846083BF83B7816083BF7894889574
:1040A00083B78E7F83BF0FB6F894A8958091600088
:1040B000886180936000109260000FBE08950E9496
:1040C000EC070C94B10382E084BD93E095BD9AEFB8
:1040D00097BD80936E0008952FB7F89480911903CF
:1040E00090911A03A0911B03B0911C032FBF089558
:1040F0002FB7F8946091190370911A0380911B03F4
:1041000090911C032FBF08959C014FB7F8948091A4
:10411000190390911A03A0911B03B0911C034FBF88
:10412000821B930B089578941F920F920FB60F92F3
:1041300011248F939F93AF93BF9380911903909114
:104140001A03A0911B03B0911C030196A11DB11D80
:104150008093190390931A03A0931B03B0931C033D
:10416000BF91AF919F918F910F900FBE0F901F90B5
:10417000189581E08093E00080E28093D80010924F
:10418000C9008FE19EE40197F1F700C0000087E0CD
:1041900090EBDC0180932A0390932B03A0932C03D4
:1041A000B0932D039CE088E10FB6F894A895809316
:1041B00060000FBE90936000FFCF8091CB02089506
:1041C0000895CF93DF9320912301222339F020918A
:1041D000CD0227FF03C060E222E002C068E021E0D8
:1041E0002093E9002FEF3091E800215035FD06C003
:1041F00035ED3A95F1F700002111F5CF2091E80057
:1042000025FF1DC0EC0180912301811105C040E014
:1042100050E068E070E003C070E040E050E0CE01A4
:104220000E9402238091E8008E778093E80080E26C
:10423000FE01ABEAB2E001900D928A95E1F7DF91C1
:10424000CF9108958093A8027093AA026093A90267
:1042500080912103843001F582E08093E9008FEFA3
:104260009091E800815095FD06C095ED9A95F1F783
:1042700000008111F5CF8091E80085FF0DC040E07E
:1042800050E063E070E088EA92E00E9402238091AF
:10429000E8008E778093E8000895BC0184E00C94D8
:1042A0002221BC0183E00C942221089580912003F7
:1042B000811109C00E9493240E94F0248091E200A1
:1042C00084608093E20008951092200308950C9476
:1042D000E81F60911D0381E0611101C080E00C9432
:1042E000D31F9091210381E0943009F080E0609128
:1042F0001D030C94D81F42E061EC81E00E940C2465
:1043000042E261EC82E00E940C249091210381E062
:10431000943009F080E060911D030C94E11F8091BE
:104320002303833009F461C030F4813071F08230AE
:1043300009F49AC008958A3009F486C08B3009F4D4
:104340006CC0893009F0A8C020C080912203813A56
:1043500009F0A2C08091E800877F8093E8008091F7
:10436000260390912703892B21F460E28BEA92E0E7
:1043700003C060E080E090E070E00E944D238091F7
:10438000E8008B778093E8000895809122038132C2
:1043900009F082C08091260390912703029708F0CC
:1043A0007BC08091E800877F8093E8008091E800DF
:1043B00082FD05C0809121038111F8CF6DC020914D
:1043C000F3008091F20090E0922B029731F48091FB
:1043D000F100813011F0863021F48091F10080935A
:1043E000CB028091E8008B7753C080912203813A01
:1043F00009F052C08091260390912703892B09F080
:104400004BC08091E800877F8093E8008091E800AE
:1044100080FFFCCF8091230136C08091220381323E
:10442000D9F58091260390912703892BA9F58091D6
:10443000E800877F8093E8000E9441248091240354
:10444000809323010C94EC0780912203813221F5A3
:104450008091E800877F8093E8000E94412480914A
:1044600025038093CC02089580912203813AA1F420
:104470008091E800877F8093E8008091E80080FFCA
:10448000FCCF8091CC028093F1008091E8008E7780
:104490008093E8000C944124089584B7877F84BFFB
:1044A0000FB6F894A89580916000886180936000B1
:1044B000109260000FBE90E080E80FB6F8948093F1
:1044C0006100909361000FBE0C94E31F0E9493243F
:1044D0000E94F024E2EEF0E0808184608083789492
:1044E0000C94852787E191E00C94BB1E80912103F9
:1044F0008530A9F480912103853079F40E9434201D
:1045000080911F038823B1F30E94F51F882391F344
:104510000E94EC220E94EC07EDCF0C945F200895DE
:1045200008950C949322292F332723303105C9F0A5
:1045300060F42130310581F02230310509F044C0AA
:104540008BE390E029E534E043C021323105E1F00E
:104550002232310549F138C082E190E024E934E0AB
:1045600037C099278130910549F028F0029761F50D
:10457000EFE2F4E005C0E5E5F4E002C0E5E4F4E0D4
:10458000849190E09F0124C06115710541F0613074
:104590007105D1F489E090E024E834E019C089E0A5
:1045A00090E02BE634E014C06115710541F06130F4
:1045B000710551F48DE690E026EA34E009C080E40C
:1045C00090E023E135E004C080E090E020E030E0BE
:1045D000FA0131832083089580E189BD82E189BD9C
:1045E00009B400FEFDCF8091D8008F7D8093D80064
:1045F0008091E00082608093E0008091E00081FD86
:10460000FCCF0895CF92DF92EF92FF920F931F930A
:10461000CF93DF93EC018B017A010E94602481111A
:1046200033C0E114F10439F0F70180819181081B56
:10463000190BC80FD91FC12CD12C0115110519F167
:104640008091E80085FD16C08091E8008E77809308
:10465000E800E114F10449F0F70180819181C80E6E
:10466000D91ED182C08285E00FC00E9460248823B9
:1046700021F30AC089918093F10001501109FFEFE5
:10468000CF1ADF0ADACF80E0DF91CF911F910F912F
:10469000FF90EF90DF90CF90089520912803309104
:1046A00029032617370748F06115710539F4209161
:1046B000E8002E772093E80001C0B901FC0120E05A
:1046C0006115710579F1809121038823F1F185301D
:1046D000F1F18091E80083FD3CC08091E80082FD0B
:1046E0002EC08091E80080FFEBCF2091F3008091F5
:1046F000F20090E0922B6115710551F08830910520
:1047000038F421912093F100615071090196F3CFA3
:1047100021E0089709F020E08091E8008E778093EF
:10472000E800CECF2111CFCF0AC08091210388238A
:1047300061F0853061F08091E80083FD0AC08091CE
:10474000E80082FFF2CF80E0089582E0089583E0E0
:10475000089581E0089520912803309129032617B8
:10476000370748F06115710539F42091E8002E777C
:104770002093E80001C0B901FC0120E0611571053A
:1047800091F180912103882309F440C0853009F418
:104790003FC08091E80083FD3DC08091E80082FD2C
:1047A0002FC08091E80080FFE9CF2091F300809135
:1047B000F20090E0922B6115710559F08830910557
:1047C00040F424912093F1003196615071090196D3
:1047D000F2CF21E0089709F020E08091E8008E7781
:1047E0008093E800CBCF2111CCCF0AC08091210368
:1047F000882361F0853061F08091E80083FD0AC074
:104800008091E80082FFF2CF80E0089582E0089571
:1048100083E0089581E00895982F973068F590938C
:10482000E900981739F07091EC002091ED0050915B
:10483000F00003C0242F762F50E021FD02C09F5FBF
:10484000ECCF3091EB003E7F3093EB003091ED00E8
:104850003D7F3093ED003091EB0031603093EB0001
:104860007093EC002093ED005093F0002091EE0047
:1048700027FDE5CF80E008958F708093E90081E007
:1048800008958091220387FF11C08091E80082FD86
:1048900005C0809121038111F8CF11C08091E800FB
:1048A0008B770BC080912103882349F08091E80029
:1048B00080FFF8CF8091E8008E778093E80008951C
:1048C0002091E4003091E50095E64091EC00842FC2
:1048D000817040FF23C08091E80080FD1DC0809161
:1048E0002103882399F0853099F08091EB0085FDB4
:1048F00011C04091E4005091E5002417350729F3D9
:10490000915011F09A01E1CF84E0089582E008957A
:1049100083E0089581E0089580E008954091E800E3
:1049200042FFDDCF08950E9401250E940925E0EE97
:10493000F0E0808181608083E8EDF0E080818F7716
:10494000808319BCA7EDB0E08C918E7F8C93808121
:104950008F7E80831092200308950F931F93CF932F
:10496000DF930E9401250E940925C8EDD0E08881CF
:104970008F77888388818068888388818F7D88830A
:1049800019BC1092210310921D0310921F03109264
:104990001E0300EE10E0F80180818B7F8083888108
:1049A0008160888342E060E080E00E940C24E1EEB8
:1049B000F0E080818E7F8083E2EEF0E08081816094
:1049C0008083808188608083F80180818E7F8083EE
:1049D000888180618883DF91CF911F910F91089525
:1049E000E8EDF0E080818F7E8083E7EDF0E080816C
:1049F0008160808384E082BF81E0809320030C94F7
:104A0000AD24E8EDF0E080818E7F80831092E2009B
:104A100008951092DA001092E10008951F920F920B
:104A20000FB60F9211242F933F934F935F936F9381
:104A30007F938F939F93AF93BF93EF93FF93809157
:104A4000E10082FF0BC08091E20082FF07C08091ED
:104A5000E1008B7F8093E1000E9484278091DA003F
:104A600080FF1FC08091D80080FF1BC08091DA00BA
:104A70008E7F8093DA008091D90080FF0DC080E1A5
:104A800089BD82E189BD09B400FEFDCF81E080933C
:104A900021030E94562105C019BC109221030E94D7
:104AA00064218091E10080FF19C08091E20080FFC5
:104AB00015C08091E2008E7F8093E2008091E20039
:104AC00080618093E2008091D80080628093D8005A
:104AD00019BC85E0809321030E9469218091E10047
:104AE00084FF30C08091E20084FF2CC080E189BD4A
:104AF00082E189BD09B400FEFDCF8091D8008F7D91
:104B00008093D8008091E1008F7E8093E1008091B6
:104B1000E2008F7E8093E2008091E20081608093CA
:104B2000E20080911D03882311F084E007C080918A
:104B3000E30087FD02C081E001C083E08093210390
:104B40000E9471218091E10083FF29C08091E200E1
:104B500083FF25C08091E100877F8093E10082E0A0
:104B60008093210310921D038091E1008E7F80933A
:104B7000E1008091E2008E7F8093E2008091E2006C
:104B800080618093E20042E060E080E00E940C24BB
:104B90008091F00088608093F0000E946721FF916F
:104BA000EF91BF91AF919F918F917F916F915F91A5
:104BB0004F913F912F910F900FBE0F901F9018951E
:104BC0001F920F920FB60F9211242F933F934F9382
:104BD0005F936F937F938F939F93AF93BF93CF9385
:104BE000DF93EF93FF93C091E900CF708091EC00C9
:104BF000D82FD17080FDD0E81092E9008091F000AC
:104C0000877F8093F00078940E9424261092E90018
:104C10008091F00088608093F000CD2BCF70C0931E
:104C2000E900FF91EF91DF91CF91BF91AF919F91FB
:104C30008F917F916F915F914F913F912F910F9045
:104C40000FBE0F901F9018951F93CF93DF93CDB792
:104C5000DEB7AA970FB6F894DEBF0FBECDBFE2E273
:104C6000F3E08091F100819323E0EA32F207C9F783
:104C70000E948F218091E80083FF2EC18091220342
:104C800090912303492F50E04A30510508F024C188
:104C9000FA01EE59FF4F0C94FA27803821F0823840
:104CA00009F01AC108C080911E0390911F03992337
:104CB00089F082600FC0809126038F70873008F0E2
:104CC0000BC18093E9008091EB0085FB882780F978
:104CD0001092E9009091E800977F9093E80080930C
:104CE000F1001092F100D1C0282F2D7F09F0F4C0FF
:104CF000882319F0823061F0EFC080912403813065
:104D000009F0EAC0933009F080E080931F032EC0C1
:104D10008091240381112AC0809126038F702FEF88
:104D2000280F263008F0D8C08093E9002091EB00CE
:104D300020FF1CC0933021F48091EB00806214C0EE
:104D40009091EB0090619093EB0021E030E0A9019D
:104D500002C0440F551F8A95E2F74093EA00109273
:104D6000EA008091EB0088608093EB001092E900EC
:104D70008091E800877F8093E8000E944124ACC0C6
:104D80008111AAC0109124031F778091E3008078DD
:104D9000812B8093E3008091E800877F8093E80077
:104DA0000E9441248091E80080FFFCCF8091E300C5
:104DB00080688093E300111102C082E001C083E0AB
:104DC0008093210389C08058823008F085C080918B
:104DD0002403909125038C3D53E0950779F583E0FA
:104DE0008A838AE289834FB7F894DE01139620E024
:104DF0003EE051E2E32FF0E050935700E49120FFB2
:104E000003C0E295EF703F5FEF708E2F90E0EA30C5
:104E100010F0C79601C0C0968D939D932F5F2431EB
:104E200049F74FBF8091E800877F8093E8006AE2EE
:104E300070E0CE0101960E944D2316C060912603BA
:104E400070912703AE014F5F5F4F0E949122BC011A
:104E5000892B09F441C09091E800977F9093E80076
:104E600089819A810E94AB238091E8008B7780939F
:104E7000E80032C0803881F58091E800877F809318
:104E8000E80080911D038093F1008091E8008E7707
:104E900072CF811121C0809124039091250399271D
:104EA0000297D4F48091E800877F8093E800809196
:104EB000240380931D030E94412480911D038111CE
:104EC00006C08091E30087FD02C081E001C084E05C
:104ED000809321030E947B218091E80083FF0AC018
:104EE0008091E800877F8093E8008091EB008062EA
:104EF0008093EB00AA960FB6F894DEBF0FBECDBF2D
:104F0000DF91CF911F9108950895CF938091210350
:104F10008823A1F0C091E900CF709091EC00892F17
:104F2000817090FD80E8C82B1092E9008091E80024
:104F300083FD0E942426CF70C093E900CF9108958D
:104F4000DB018F939F930E941E28BF91AF91A29F78
:104F5000800D911DA39F900DB29F900D1124089577
:104F6000AA1BBB1B51E107C0AA1FBB1FA617B7078F
:104F700010F0A61BB70B881F991F5A95A9F78095AB
:104F80009095BC01CD01089597FB072E16F400946F
:104F900007D077FD09D00E94B02707FC05D03EF46A
:104FA000909581959F4F0895709561957F4F0895D5
:104FB000A1E21A2EAA1BBB1BFD010DC0AA1FBB1F1D
:104FC000EE1FFF1FA217B307E407F50720F0A21B8F
:104FD000B30BE40BF50B661F771F881F991F1A94FC
:104FE00069F760957095809590959B01AC01BD0126
:104FF000CF010895EE0FFF1F0590F491E02D099465
:105000000E940828332312F48A1B9B0B0C94192846
:10501000A29FB001B39FC001A39F700D811D1124F9
:10502000911DB29F700D811D1124911D08950E9444
:105030000828B7FF0895821B930B08950E94082843
:10504000A59F900DB49F900DA49F800D911D1124DC
:105050000895B7FF0C941E280E941E28821B930BF4
:105060000895FC014150504030F001900616D1F7F0
:105070003197CF010895882799270895FB01DC0116
:1050800004C08D910190801921F441505040C8F71F
:10509000881B990B0895F999FECF92BD81BDF89AAE
:1050A000992780B50895A6E1B0E044E050E00C9463
:1050B0008528A8E1B0E042E050E00C948528262F36
:1050C000F999FECF92BD81BDF89A019700B40216FE
:1050D00039F01FBA20BD0FB6F894FA9AF99A0FBEAC
:1050E00008950396272F0E9460280E945F28252F8D
:1050F0000E946028242F0C9460280196272F0E947C
:1051000060280C945F28DC01CB01FC01F999FECFEB
:1051100006C0F2BDE1BDF89A319600B40D9241503F
:0A5120005040B8F70895F894FFCF4F
:10512A00C8005802010102001000101001191A1BD0
:10513A001C1D1E1F202122DD20E120552151214D59
:10514A0021E02001E200E900EA00B500B600B7005C
:10515A00CD008301CC008A0192019401210223022D
:10516A0024022502260227022A02B300B4006F0095
:10517A007000818283E200E900EA00B500B600B758
:10518A0000CD008301CC008A0192019401210223FF
:10519A000224022502260227022A02B300B4006F63
:1051AA000070008182836667F7F1C63231963497C0
:1051BA00949593929190F6F5F4F03600010202026A
:1051CA00020606060909090909090F0F0F0F0F0F31
:1051DA00151515181919191919191919191923242D
:00000001FF
